******************************************************************************
               TMS320C6x Linker Unix v7.4.0                    
******************************************************************************
>> Linked Mon Nov 19 18:19:13 2012

OUTPUT FILE NAME:   <../bin/pcieboot_localreset_evm6670l.out>
ENTRY POINT SYMBOL: "_c_int00"  address: 008f8000


MEMORY CONFIGURATION

         name            origin    length      used     unused   attr    fill
----------------------  --------  ---------  --------  --------  ----  --------
  L2_LOCAL              008f2dc0   0000d240  00000bac  0000c694  RW X


SEGMENT ALLOCATION MAP

run origin  load origin   length   init length attrs members
----------  ----------- ---------- ----------- ----- -------
008f2dc0    008f2dc0    00000700   00000700    r-x
  008f2dc0    008f2dc0    00000700   00000700    r-x .text
008f34c0    008f34c0    00000400   00000000    rw-
  008f34c0    008f34c0    00000400   00000000    rw- .stack
008f38c0    008f38c0    0000000c   0000000c    rw-
  008f38c0    008f38c0    0000000c   0000000c    rw- .fardata
008f38cc    008f38cc    00000020   00000020    r--
  008f38cc    008f38cc    00000020   00000020    r-- .cinit
008f8000    008f8000    00000080   00000080    r-x
  008f8000    008f8000    00000080   00000080    r-x .text:_c_int00


SECTION ALLOCATION MAP

 output                                  attributes/
section   page    origin      length       input sections
--------  ----  ----------  ----------   ----------------
.text      0    008f2dc0    00000700     
                  008f2dc0    00000180     rts6600_elf.lib : copy_decompress_rle.obj (.text:__TI_decompress_rle_core)
                  008f2f40    00000100                     : autoinit.obj (.text:_auto_init_elf)
                  008f3040    00000100                     : cpy_tbl.obj (.text:copy_in)
                  008f3140    000000c0                     : exit.obj (.text:exit)
                  008f3200    000000c0                     : tls.obj (.text:tls:init:__TI_tls_init)
                  008f32c0    000000a0                     : memcpy64.obj (.text:memcpy)
                  008f3360    00000060                     : cpp_init.obj (.text:__TI_cpp_init)
                  008f33c0    00000060     pcieboot_localreset.obj (.text)
                  008f3420    00000040     rts6600_elf.lib : args_main.obj (.text:_args_main)
                  008f3460    00000020                     : exit.obj (.text:abort)
                  008f3480    00000020                     : copy_decompress_none.obj (.text:decompress:none:__TI_decompress_none)
                  008f34a0    00000020                     : copy_decompress_rle.obj (.text:decompress:rle24:__TI_decompress_rle24)

.stack     0    008f34c0    00000400     UNINITIALIZED
                  008f34c0    00000008     rts6600_elf.lib : boot.obj (.stack)
                  008f34c8    000003f8     --HOLE--

.fardata   0    008f38c0    0000000c     
                  008f38c0    0000000c     rts6600_elf.lib : exit.obj (.fardata)

.cinit     0    008f38cc    00000020     
                  008f38cc    0000000d     (.cinit..fardata.load) [load image, compression = rle]
                  008f38d9    00000003     --HOLE-- [fill = 0]
                  008f38dc    00000008     (__TI_handler_table)
                  008f38e4    00000008     (__TI_cinit_table)

.text:_c_int00 
*          0    008f8000    00000080     
                  008f8000    00000080     rts6600_elf.lib : boot.obj (.text:_c_int00)


LINKER GENERATED COPY TABLES

__TI_cinit_table @ 008f38e4 records: 1, size/record: 8, table size: 8
	.fardata: load addr=008f38cc, load size=0000000d bytes, run addr=008f38c0, run size=0000000c bytes, compression=rle


LINKER GENERATED HANDLER TABLE

__TI_handler_table @ 008f38dc records: 2, size/record: 4, table size: 8
	index: 0, handler: __TI_decompress_rle24
	index: 1, handler: __TI_decompress_none


GLOBAL SYMBOLS: SORTED ALPHABETICALLY BY Name 

address    name
--------   ----
008f3460   C$$EXIT
008f38e4   __TI_CINIT_Base
008f38ec   __TI_CINIT_Limit
008f38dc   __TI_Handler_Table_Base
008f38e4   __TI_Handler_Table_Limit
UNDEFED    __TI_INITARRAY_Base
UNDEFED    __TI_INITARRAY_Limit
008f38c0   __TI_STACK_END
00000400   __TI_STACK_SIZE
00000000   __TI_STATIC_BASE
UNDEFED    __TI_TLS_INIT_Base
UNDEFED    __TI_TLS_INIT_Limit
00000001   __TI_args_main
008f3360   __TI_cpp_init
008f3480   __TI_decompress_none
008f34a0   __TI_decompress_rle24
008f38c8   __TI_enable_exit_profile_output
ffffffff   __TI_pprof_out_hndl
ffffffff   __TI_prof_data_size
ffffffff   __TI_prof_data_start
008f3200   __TI_tls_init
ffffffff   __binit__
ffffffff   __c_args__
008f3420   _args_main
008f2f40   _auto_init_elf
008f8000   _c_int00
008f38c0   _cleanup_ptr
008f38c4   _dtors_ptr
008f34c0   _stack
008f3460   abort
ffffffff   binit
008f3040   copy_in
008f3140   exit
008f33f8   main
008f32c0   memcpy
008f33c0   start_boot


GLOBAL SYMBOLS: SORTED BY Symbol Address 

address    name
--------   ----
00000000   __TI_STATIC_BASE
00000001   __TI_args_main
00000400   __TI_STACK_SIZE
008f2f40   _auto_init_elf
008f3040   copy_in
008f3140   exit
008f3200   __TI_tls_init
008f32c0   memcpy
008f3360   __TI_cpp_init
008f33c0   start_boot
008f33f8   main
008f3420   _args_main
008f3460   C$$EXIT
008f3460   abort
008f3480   __TI_decompress_none
008f34a0   __TI_decompress_rle24
008f34c0   _stack
008f38c0   __TI_STACK_END
008f38c0   _cleanup_ptr
008f38c4   _dtors_ptr
008f38c8   __TI_enable_exit_profile_output
008f38dc   __TI_Handler_Table_Base
008f38e4   __TI_CINIT_Base
008f38e4   __TI_Handler_Table_Limit
008f38ec   __TI_CINIT_Limit
008f8000   _c_int00
ffffffff   __TI_pprof_out_hndl
ffffffff   __TI_prof_data_size
ffffffff   __TI_prof_data_start
ffffffff   __binit__
ffffffff   __c_args__
ffffffff   binit
UNDEFED    __TI_INITARRAY_Base
UNDEFED    __TI_INITARRAY_Limit
UNDEFED    __TI_TLS_INIT_Base
UNDEFED    __TI_TLS_INIT_Limit

[36 symbols]
